:1000000012C018951895189518955AC192C118954F
:100010001895189518951895189518951895189578
:100020001895189518958FED8DBFC0ECE8EB4E2E06
:10003000DD275D2EEEE7F0E0A0E6B0E088278D93A7
:100040003197E9F7EDD166248C9A85E083BF80E093
:1000500080BF80E08FBD87E08EBD789489B78260D5
:1000600089BF89B7806889BFBED1CED1ECECF6E0FC
:10007000B2D1B7D1ECEDF6E0AED18CE019D2E2E02E
:10008000F0E0C5D1949880E08093520080E090E049
:1000900090934D0080934C0000E010E020E030E0B1
:1000A000A4E60D931D932D933C9300E010E020E017
:1000B00030E0A8E60D931D932D933C934BE450E064
:1000C00060E070E0A4E60D911D912D913C917AD2F3
:1000D00014F009F002C00000F1CFEF93FF93E8E2C3
:1000E000FCE44CD2FF91EF91949A89B78D7F89BF40
:1000F00089B78F7789BFA8E60D911D912D913C910D
:1001000040E050E061E070E0F3D1A0E60D931D9374
:100110002D933D93A0E60D911D912D913C91ACE462
:100120004D915C916627772748D2ACE60D931D93DD
:100130002D933D9358D18FE711E064D1A0E7ECE611
:10014000F0E056D240E452E46FE070E0ACE60D918E
:100150001D912D913C9136D20CF001C002C045C0DA
:100160002DC040EA56E861E070E0ACE60D911D91CB
:100170002D913C9127D20CF001C002C04DC01EC091
:1001800040E157E260E070E0ACE60D911D912D91E9
:100190003C9118D20CF001C002C055C00FC048EE0F
:1001A00053E060E070E0ACE60D911D912D913C9123
:1001B00009D214F009F001C001C05CC007E00F9340
:1001C000A0E77ED2482F0F91041BA1E80C938FE784
:1001D000A1E81C9117D1A0EAB0E0ECE6F0E008D26B
:1001E000F2D0EAEEF6E0F7D05FC0E0E7F0E001E041
:1001F000A8E75ED282E0E0E7F0E004E00A93ACE733
:1002000050D2A8E7E2D0EEEEF6E0E5D0ACE7DDD0E4
:10021000E0EFF6E0E0D048C0E0E7F0E003E0A8E778
:1002200047D284E0E0E7F0E002E00A93ACE739D29D
:10023000A8E7CBD0EEEEF6E0CED0ACE7C6D0E6EF46
:10024000F6E0C9D031C0E0E7F0E002E0A8E730D244
:1002500083E0E0E7F0E003E00A93ACE722D2A8E70E
:10026000B4D0EEEEF6E0B7D0ACE7AFD0E6EFF6E014
:10027000B2D01AC0E0E7F0E001E0A8E719D282E0CE
:10028000E0E7F0E004E00A93ACE70BD2ECEFF6E035
:10029000A2D0A8E79AD0EEEEF6E09DD0ACE795D0DC
:1002A000E6EFF6E098D000C08FEB11E0ABD08CE029
:1002B000FFD089B7826089BF89B7806889BFE2CEE5
:1002C0000F921F922F923F924F925F927F92AF9226
:1002D000BF920F931F932F933F934F935F936F930F
:1002E0007F938F939F93AF93BF93CF93DF93EF93BE
:1002F000FF938FB78F93A8E657D08F918FBFFF9151
:10030000EF91DF91CF91BF91AF919F918F917F91AD
:100310006F915F914F913F912F911F910F91BF90DE
:10032000AF907F905F904F903F902F901F900F90D5
:1003300018950F921F922F923F924F925F927F9249
:10034000AF92BF920F931F932F933F934F935F935F
:100350006F937F938F939F93AF93BF93CF93DF93CD
:10036000EF93FF938FB78F93A4E61ED08F918FBF2B
:10037000FF91EF91DF91CF91BF91AF919F918F91BD
:100380007F916F915F914F913F912F911F910F91AD
:10039000BF90AF907F905F904F903F902F901F90B5
:1003A0000F901895F894FFCF0D911D912D913C91D0
:1003B00081E0080F8827181F281F381F3C932E93B1
:1003C0001E930E930895A0EAB0E08D91882311F05A
:1003D00069D0FBCF0895EDD0802D11F063D0FBCF15
:1003E000089580EC65C081E063D017D080E860C0DC
:1003F0008FE7213039F08FEB223021F08FE8233066
:1004000009F08FEC810F54C080E852D0089588EE37
:1004100093E0C0D03197D9F7089583E09927BAC007
:100420008AEF90E0B7D08E9AB89AB99ABA9ABB9AE6
:10043000BC9AC49885E090E0ADD0C3989698C098D7
:10044000C19AC29AC39AEF93FF93E0EFF1E096D07E
:10045000FF91EF91C3989BD0C39AEF93FF93E0EF86
:10046000F1E08CD0FF91EF91C39891D0C39AEF93B4
:10047000FF93E0EFF1E082D0FF91EF91C39887D036
:10048000C298C39AEF93FF93E0EFF1E077D0FF912A
:10049000EF91C3987CD088E20BD08EE009D086E043
:1004A00007D00895C49A829505D004D070D00895DD
:1004B000C498F9CF859510F4C29A01C0C298859569
:1004C00010F4C19A01C0C198859510F4C09A01C07A
:1004D000C098859510F4969A01C09698C39AEF93A8
:1004E000FF93E0EFF1E04AD0FF91EF91C3980895B8
:1004F00022D006D000FC01D0089528D030D0089535
:10050000842F952FA62FB72F4427552766277727A7
:10051000F1E2889409C020F4480F591F6A1F7B1F1D
:10052000769567955795479537952795179507952C
:10053000FA9589F708950024E89477FF02C006D061
:10054000689400F809D010F80124089512D04F5F84
:100550005F4F6F4F7F4F0895E89437FF08950095E0
:100560001095209530950F5F1F4F2F4F3F4F689488
:100570000895409550956095709508953197F1F7DD
:100580000895689462F80895E89462F8089581E007
:1005900090E000C0EF93FF93EE27E82BE92B31F0BA
:1005A000E8E8F3E13197F1F70197D1F7FF91EF9187
:1005B0000895C895319600200895040F151F261F31
:1005C000371F089504171507260737070895000FEA
:1005D000111F221F331F0895009510952095309507
:1005E0000F5F1F4F2F4F3F4F0895019110810EC095
:1005F00001911191219130810BC00191108117FF60
:1006000005C03FEF2FEF04C00081112722273327B9
:1006100037FF03C0E1DF8DE28D93CF93DF93CF925D
:10062000DF92EF92AA24BB24CC24DD24EE2440E206
:10063000CAE0DD2755E093E38881890F87FD9F702D
:1006400083FD907F891B89935A95A9F7C0DFAA1C67
:10065000BB1CCC1CDD1CEE1C4A9551F7E894EFE066
:10066000FF2782910ED0EB30E0F71EF068948A2DC0
:100670000CD088278D93EF90DF90CF90DF91CF91B2
:100680000895982F829501D0892F8F70805D26F074
:10069000803309F4089568948D93089588278D9385
:1006A000089509919191992351F08A95D9F731973D
:1006B00081918D930A9519F08823D1F70895EECF93
:1006C0008FEF83959D919923E1F70895206E7578BA
:1006D000696573686F702E636F6D0000202020467F
:1006E000756E20436F756E74000020487A002E00EE
:0E06F000204D487A0000204B487A0000200080
:00000001FF
